:100000008A110A120528000009000730990083169A
:10001000051085100511851605168312E830A0001D
:100020000330A1007922AF010130B5001321851AF8
:1000300026283508013C031D1F283A21B5011F3031
:100040008305051E242867201F3083051F30830584
:10005000851E33283508003C031D31282921013035
:10006000B5001F3083051F3083056430A000A10157
:1000700079223208013EB20032080A3C031D4428AE
:10008000B2013308013EB3001F30830533083C3C06
:10009000031D4E28B3013408013EB4001F30830510
:1000A00034080F3C031D63282F08003C031D5A2809
:1000B00013215E281F308305FD20AF011F3083050B
:1000C000B401B301B2011F30830517286628051457
:1000D0000130AF00B0010130B100B201B301B40191
:1000E0003108013C031DE528B101AC012C08323C6C
:1000F000031C8428051E7E280130B1001F308305B3
:100100000130AC07031C76281F3083059630A00011
:10011000A10179223208023EB20032080A3C031DD6
:100120009528B2013308013EB3001F308305330820
:100130003C3C031D9F28B3013408013EB4001F302E
:100140008305AC012C08323C031CB028051EAA28EC
:100150000130B1001F3083050130AC07031CA22819
:100160001F3083053008003C031DC4283408043CBC
:10017000031DC228292105100130B0000E30B40043
:100180003730B3001F3083051F308305AC012C08C6
:10019000323C031CD528051ECF280130B1001F308A
:1001A00083050130AC07031CC7281F3083053408C2
:1001B000033C031DE228FD20051467220510B4014D
:1001C000B301B2011F30830570281F3083052C3026
:1001D000A0000130A10079223308003C0318F12867
:1001E00074211F3083053230A000A101792205104F
:1001F0000E30B4002D30B30008000514F430A00018
:100200000130A10079222F22872121229B21212246
:10021000D521212291212122872121224E212F2205
:100220002F22051008000514F430A0000130A100B1
:1002300079222F22872121229B212122D5212122AF
:1002400091212122872121224E212F222F220510A8
:1002500008000514F430A0000130A10079222F22FB
:100260008C212122912121229921212267222F22D2
:10027000051008000514F430A0000130A100792217
:100280002F228C212122912121229F2121226722AC
:100290002F2205100800452256220800562245222A
:1002A00045224522080056224522562245220800B2
:1002B00056224522452208004522080045224522B3
:1002C0005622452208005622562245220800452281
:1002D00045224522452208004522452208004522A4
:1002E000562256225622080056224522562208003F
:1002F0004522562245224522080056225622080051
:10030000562245220800562256225622080045222F
:1003100056225622452208005622562245225622AF
:100320000800452256224522080045224522452242
:100330000800562208004522452256220800452280
:100340004522452256220800452256225622080000
:100350005622452245225622080056224522562280
:1003600056220800562256224522452208005622CF
:10037000562256225622562208004522562256223E
:10038000562256220800452245225622562256223F
:1003900008004522452245225622562208004522C1
:1003A0004522452245225622080045224522452263
:1003B0004522452208005622452245224522452253
:1003C0000800562256224522452245220800562280
:1003D00056225622452245220800562256225622EF
:1003E0005622452208004522562245225622452201
:1003F00056220800562256224522452256225622CF
:100400000800452245225622562245224522080050
:1004100056224522452256224522080056224522D0
:1004200045224522562208005622452245224522D1
:1004300045225622080005113C30A000A101792276
:10044000080005113C30A000A10179223C30A00039
:10045000A10179223C30A000A101792208000511F8
:100460003C30A000A10179223C30A000A1017922FA
:100470003C30A000A10179223C30A000A1017922EA
:100480003C30A000A1017922080005150530840048
:100490000230AA007030A0000230A1003030A2006B
:1004A0000030A300B42205111B22080005150530F9
:1004B00084000230AA007030A0000230A100C030D9
:1004C000A2000030A300B42205111B22080005156C
:1004D000053084000230AA007030A0000230A10074
:1004E000B030A2000430A300B42205111B22080082
:1004F000782AA0080319842A8B22A0030000000098
:10050000000000000000792AA108031908008B22CE
:10051000A103A003792A0C30A500A50B8D2A0000A9
:1005200000001230A200A20B9A2A9C229C220000FA
:10053000000008009C22932A0D30A400A40B9E2AE0
:10054000000008001030A8020001031C013EA902AF
:10055000031C0800AB2A0A30A8020001031C013E5C
:10056000A902031C0800AB2A2A0880042008A8005E
:100570002108A900A2220130A202031CA3032A0918
:1005800080052008A8002108A900A222A208031DB6
:0A059000B42AA308031DB42A0800D2
:02400E00C433B9
:00000001FF
